:100000000C94C1010C94E0010C94E0010C94E0010B
:100010000C94E0010C94E0010C94E0010C94E001DC
:100020000C94E0010C94E0010C94911A0C94671B61
:100030000C94B4150C94E0010C94E0010C94E001D4
:100040000C94E0010C94E0010C94E0010C94E001AC
:100050000C94E0010C943C160C94E0010C94E0012B
:100060000C94E0010C94E0010C94E0010C94E0018C
:100070000C94E0010C94E0010C94E0010C94E0017C
:100080000C94E0010C94E0010C94E0010C94E0016C
:100090000C94E0010C94E001E203E2030E040E0470
:1000A000830583058305830576040F052005200558
:1000B000D812CE12DB12231327132713231327136F
:1000C0002713FC12271306131013271327132713C4
:1000D000271323132713271323132713E912271397
:1000E0002713201320132013201320132013201371
:1000F0002013201325132713D812CB1227132713ED
:10010000271327132713271327132713271327131F
:10011000251327132713231327131E131E131E1330
:100120001E131E131E131E131E131E132513D81B7E
:10013000FF1BF71CFF1BF71C4B1C6E1CF71CC51C80
:10014000D41C290000003A003B003C003D003E006A
:100150003F004000410042004300440045004C0085
:1001600035001E001F002000210023002400250070
:10017000260027002D002E002A002B0014001A0054
:1001800008001500170022001C0018000C001200C7
:1001900013002F003100E0000400160007000900E2
:1001A0000A00E1010B000D000E000F0033003400C7
:1001B00028714A621D001B000600190005002A0074
:1001C0001100100036003700380030004B724D61CE
:1001D00000000000E20000002C0028002C4100007C
:1001E000E60065000000E7004E710100000001001C
:1001F00001000100010001000100010001000100F7
:1002000001000100005C010001000100010001008B
:1002100001000100010001000100010001000100D6
:1002200001000100010001000100010001000100C6
:1002300001000100010001000100010001000100B6
:10024000010001000100010001000100280052002E
:100250002A0001000100010001000100010001006D
:100260000100010001000100500051004F00010099
:100270000100010001000100010001000100000077
:100280000100490001000000010001000000010020
:1002900001000C037A004500720067006F00000047
:1002A000140347007200650065006E004A0061009B
:1002B00063006B0000000403090409023B00020113
:1002C00000A0FA0904000001030101000921110145
:1002D0000001224000070581030800010904010014
:1002E0000103000000092111010001223B00070564
:1002F00082032000011201000200000008EDFE2B25
:10030000B901000102000105010906A101850605E8
:100310000719E029E71500250195087501810205F7
:1003200007190029EF1500250195F07501810205D7
:10033000081901290595057501910295017503912B
:1003400001C005010906A101050719E029E715000B
:100350002501950875018102950175088101050740
:10036000190029FF150026FF009506750881000574
:1003700008190129059505750191029501750391EB
:1003800001C011241FBECFEFD0E2DEBFCDBF11E010
:10039000A0E0B1E0EAE0FBE300E00BBF02C00790A1
:1003A0000D92A632B107D9F722E0A6E2B1E001C072
:1003B0001D92A735B207E1F70E9453110C94831DDB
:1003C0000C94000081E0089581E008950C94E4010C
:1003D00008950C94E8011F93CF93DF9300D000D0D1
:1003E0001F92CDB7DEB749835A836B8330912901C1
:1003F00089819A81311114C0662359F0222349F072
:100400000E94B407182F682F89819A810E945D0786
:1004100003C00E948807182F69817A81812F04C048
:100420000E94B40769817A810F900F900F900F900E
:100430000F90DF91CF911F910C94BE0EFC01262FDF
:10044000408151816281738184810C94EB0181E050
:100450000895CF93DF93EC0160E00E941E02BE017D
:10046000DF91CF910C94E9010C9404100C940010CE
:1004700008950E9407060E9438022FEF84E39CE053
:10048000215080409040E1F700C000000C946216BB
:100490000F931F93CF93DF938C0161E00E941E02A4
:1004A000EC01B8010E94E6018823F1F1B801CE0108
:1004B0000E940D148823C1F1B801CE010E94601181
:1004C000882391F1B801CE010E946913882361F15C
:1004D000F8018281882309F1CB358DE5D807C1F079
:1004E00050F4C115FCE5DF0781F0CF3DDC45A9F4F0
:1004F0000E94EB0C19C0CC35EDE5DE0761F0CD357F
:10050000DD4559F40E942E0C08C00E9439020CC02F
:100510000E94370C02C00E943A0CC801DF91CF91B3
:100520001F910F910C94E20180E0DF91CF911F9118
:100530000F9108950E9496150C94B3020E94B60282
:100540000C949C1508950C94A20281E008950C94DB
:10055000A5020895CF93C82F0E94A3028C2F0E945A
:10056000A702CF91089580E00C94AA020E9469141A
:100570000C94AA020E94691490912801891721F015
:10058000809328010C94AA020895CF93DF93CDB7EE
:10059000DEB72B970FB6F894DEBF0FBECDBF4F83EB
:1005A000588769877A878B8761110E947A0B9E0131
:1005B0002F5F3F4F86E0F90111928A95E9F785E0B8
:1005C000FE013796D90101900D928A95E1F7898154
:1005D0009A814C815D81452B31F09F3F31F491E050
:1005E0008F3F19F403C091E001C090E090FF09C073
:1005F00049815A816B817C818D819E810E949B0AF9
:1006000005C0C9010E9427028111F2CF2B960FB6B7
:10061000F894DEBF0FBECDBFDF91CF910895FC01EE
:10062000808191810E94F6070895CF93882399F1E4
:10063000C82F8CEF8C0F813AF8F48C2F0E942D1369
:10064000811129C06C2F80910201909103010E94B9
:10065000D114882349F06C2F8091020190910301FD
:100660000E945C150E949C0B6C2F8091020190915E
:1006700003010E9451150CC080E28C0F883058F4A1
:10068000C77081E001C0880FCA95EAF70E945D0B30
:10069000CF910C949C0BCF910895882349F1682F3A
:1006A0008CEF860F813A38F480910201909103011A
:1006B0000E945C150CC080E2860F883050F4677091
:1006C00081E001C0880F6A95EAF70E94630B0C94E1
:1006D0009C0B8BE5860F833020F480E090E00C9437
:1006E0008F14685A673120F480E090E00C94A514D0
:1006F00008951F93CF93DF93182FEB010E941503EA
:10070000209741F08FE99FE00197F1F700C00000CA
:100710002197F6CF812FDF91CF911F910C944D033C
:10072000893319F060E070E002C060E570E00C947D
:100730007903882321F00E945D0B0C949C0B089593
:10074000882321F00E94630B0C949C0B0895CF9298
:10075000DF92EF92FF920F931F93CF93DF937C0171
:10076000D62FC72FFC011281058102950F700E94C0
:10077000530B8823B9F01123A9F08C2F807F80348C
:1007800021F080E28D0F883068F080912D0282FD8B
:1007900009C082E00E94FC0B0E94530B91E0D82E0E
:1007A000D92601C0D12CCC2EC2948FE0C8228C2D2A
:1007B00090E08C30910508F0A6C1FC01E45BFF4F8E
:1007C0000C942B1D8C2F807FCF70882311F0C29545
:1007D000C07F112399F0CC2309F481C180E28D0FF1
:1007E000883010F0D11104C08C2F0E945D0B03C023
:1007F0008C2F0E946D0B0E949C0B71C18D2F0E944B
:100800004D03CC2309F47FC180E28D0F883038F18D
:10081000DD2329F18C2F0E94730B24C08C2F807F45
:10082000CF70803211F0C295C07FDD2319F0D13036
:10083000A1F13DC080912D0282FF17C0112349F024
:10084000CC2329F08C2F0E945D0B0E949C0B80E032
:1008500047C180E00E944D03CC2309F454C18C2F82
:100860000E94630B0E949C0B4EC1112371F0002368
:1008700041F0013031F40E947D0B8C2B0E94850BDE
:1008800042C10E947D0B8C2B1DC0002319F001304A
:1008900009F439C10E94920B25C0112321F00630C2
:1008A00008F031C10EC0053008F02DC11BC0112366
:1008B00061F0002331F0F701858180FF10C18F7056
:1008C00085838C2F0E9499031EC1002359F0D933D0
:1008D00009F016C1FFEF07EE13E0F15000401040A1
:1008E000E1F70CC18C2F0E94A0030DC18C2F8370E7
:1008F00009F047C011110BC12D2F229526952770A5
:10090000220F220F6D2F6F70862F90E0A0E0B0E0D5
:10091000022E04C0880F991FAA1FBB1F0A94D2F78A
:10092000D4FF10C04FE050E060E070E004C0440F1E
:10093000551F661F771F2A95D2F7409550956095F1
:10094000709503C040E050E0BA01C695C695C370EB
:100950008A019B01082B192B2A2B3B2BC901B801BB
:10096000C23049F058F4C13019F00E947306CFC06C
:100970000E946106CCC00E948506C9C00E945F0625
:10098000C6C0112319F08C2F817001C08695882371
:1009900009F4BDC02D2F229526952770220F220F16
:1009A0006D2F6F70862F90E0A0E0B0E0022E04C0A3
:1009B000880F991FAA1FBB1F0A94D2F7D4FF10C03B
:1009C0004FE050E060E070E004C0440F551F661F28
:1009D000771F2A95D2F7409550956095709503C082
:1009E00040E050E0BA01C695C695C3708A019B01EC
:1009F000082B192B2A2B3B2BC901B801C23049F017
:100A000058F4C13019F00E94380781C00E942607AF
:100A10007EC00E944A077BC00E94990678C0CF70B2
:100A2000112339F08C2F0E94BF068D2F0E9499034D
:100A30006EC08D2F0E94A0038C2F0E94E00667C01D
:100A4000D23F21F128F4D03F41F0D13FC1F043C063
:100A5000D33F19F1D43F79F03EC0112341F0053066
:100A600008F051C08C2F8F710E9405074CC00630D2
:100A700008F049C0F7CF80912D0282FF18C01123E2
:100A800039F08C2F8F710E94BF063DC01123C9F32E
:100A90008C2F8F710E94E00636C0112329F08C2F15
:100AA0008F710E94AA062FC00E94A5062CC0112398
:100AB00049F0CF718C2F0E94BF0663E08C2F0E94FB
:100AC000E10B21C081E00E94FC0B0230E0F082E0EB
:100AD0000E94FC0B18C0112331F0002391F28D2FDE
:100AE0000E94150310C0002399F2D93349F41FEF77
:100AF00027EE33E0115020403040E1F700C0000005
:100B00008D2F0E944D0388EF8C0D843020F40E94BD
:100B100069140E94AA02DD20C9F00E944F0B80FDDB
:100B200015C0F70112820E94490B0E94BF06C7013F
:100B30000E94C7050E94490BDF91CF911F910F9131
:100B4000FF90EF90DF90CF900C94E006DF91CF9173
:100B50001F910F91FF90EF90DF90CF9008950F932A
:100B60001F93CF93DF93EC01688179818A810E9482
:100B700001088C010E945C070E944D06B801CE015D
:100B80000E94A703DF91CF911F910F910895CF93FA
:100B9000DF93EC01988189812B813C81232B31F0FB
:100BA0008F3F31F481E09F3F19F403C081E001C021
:100BB00080E080FD1DC0CE010E944802811110C05E
:100BC0000E94530B8823A1F08A81882389F08091A9
:100BD0002D0282FD0DC082E0DF91CF910C94FC0BC1
:100BE000CE010E94AF05CE01DF91CF910C94290276
:100BF000DF91CF9108950E947A0B0C949C0B809109
:100C00000201909103010E9467150C94FB050E945C
:100C10006A0B0C94FF0592959F70963079F010F452
:100C2000925001C09A50923068F4803F69F018F4F5
:100C3000883E40F409C0843F29F406C0883E20F075
:100C4000813F11F080E0089581E00895FC018081EA
:100C500091810E94F6070E940B060895CF93DF93BF
:100C600000D000D01F92CDB7DEB70F900F900F903D
:100C70000F900F90DF91CF910895CF93DF9300D025
:100C800000D000D0CDB7DEB726960FB6F894DEBF01
:100C90000FBECDBFDF91CF910895089508950C94B4
:100CA0004E060C944F060E945106609365017093A6
:100CB000660180936701909368010C94FB050C9486
:100CC00053060F931F9300916501109166012091C7
:100CD000670130916801602B712B822B932B1F9140
:100CE0000F910C9453060F931F930091650110917F
:100CF000660120916701309168016023712382238E
:100D000093231F910F910C9453060F931F930091FF
:100D1000650110916601209167013091680160279B
:100D20007127822793271F910F910C9453060C94DF
:100D30004E060E9497066093610170936201809352
:100D40006301909364010C94FB0560E070E0CB01BB
:100D50000C9499060F931F9341E050E060E070E01F
:100D60008A019B0104C0000F111F221F331F8A95A7
:100D7000D2F7C901B8011F910F910C9499060F93F6
:100D80001F9341E050E060E070E004C0440F551F45
:100D9000661F771F8A95D2F7809161019091620159
:100DA000A0916301B09164018A019B01082B192B6A
:100DB0002A2B3B2BC901B8011F910F910C94990666
:100DC0000F931F9341E050E060E070E004C0440FD7
:100DD000551F661F771F8A95D2F7409550956095ED
:100DE00070958091610190916201A0916301B09131
:100DF00064018A019B01082319232A233B23C9018B
:100E0000B8011F910F910C9499060F931F9341E025
:100E100050E060E070E004C0440F551F661F771F6C
:100E20008A95D2F78091610190916201A09163014E
:100E3000B09164018A019B01082719272A273B27C3
:100E4000C901B8011F910F910C9499060F931F933C
:100E50000091610110916201209163013091640160
:100E6000602B712B822B932B1F910F910C94990661
:100E70000F931F9300916101109162012091630112
:100E80003091640160237123822393231F910F917A
:100E90000C9499060F931F930091610110916201C8
:100EA0002091630130916401602771278227932785
:100EB0001F910F910C94990608952EE0929F800D3A
:100EC0001124E82FE695E695E695877051E001C07C
:100ED000550F8A95EAF785E0E89FF0011124E65D59
:100EE000FE4F20E030E070E04081CB01022E02C0D6
:100EF000969587950A94E2F78170819584278523DA
:100F0000842781932F5F3F4F2530310569F708957E
:100F10002EE0929F800D1124682F66956695669548
:100F2000982F977085E0689FB001112440E050E051
:100F300080E0FB01E40FF51FE65DFE4F208130E00D
:100F4000092E02C0369527950A94E2F721703327BF
:100F5000042E01C0220F0A94EAF7822B4F5F5F4FE5
:100F60004530510531F70895BF92CF92DF92EF924D
:100F7000FF920F931F93CF93DF938C01C090610179
:100F8000D0906201E0906301F0906401809165016E
:100F900090916601A0916701B0916801C82AD92A91
:100FA000EA2AFB2ACFE1D0E0D701C6010C2E04C00B
:100FB000B695A795979587950A94D2F780FD04C0BA
:100FC000219790F7B12C07C0BC2EB8018C2F0E943E
:100FD000D10E0197A9F38B2DDF91CF911F910F9126
:100FE000FF90EF90DF90CF90BF900895CF93DF9365
:100FF000EC010E94B407BE010E94D10EDF91CF9197
:1010000008951F93CF93DF93EB01909129019923CA
:1010100021F0CB010E94F60713C0882349F0CB01D1
:101020000E94B407182F682FCE010E945D0704C0EC
:10103000CB010E948807182FBE01812F0E94D10E7C
:10104000DF91CF911F9108951F93CF93DF93C091AC
:10105000690116E080916A01C81799F0D0E01C9FE1
:10106000F0011D9FF00D1124E559FE4F4081518183
:1010700062817381848195810E943D062196C770AB
:10108000E9CFDF91CF911F91089540919B0150913D
:101090009C0160919D0170919E0180919F019091B2
:1010A000A0010C943D06EF92FF920F931F93CF93F4
:1010B000DF938091A00182958F7009F065C08091C7
:1010C0009D01882309F460C080916901F0906A0154
:1010D00010919B0100919C0160919E0170919F0174
:1010E00091E01F3F09F090E0C0910001D091010113
:1010F000292F96E0E92E8F1509F446C06115710578
:1011000021F00F3F21F030E003C031E001C0322F69
:1011100090E030FD36C0E89EF001E99EF00D11240C
:10112000DF01A559BE4F11963C911197301329C08C
:101130003C91311326C012963C911297311121C077
:1011400013964D915C911497461B570B4C175D07F6
:10115000C0F48091A0018F7080618093A001E0595C
:10116000FE4F80818F70806180838BE991E00E94C7
:10117000C705DF91CF911F910F91FF90EF900C94D5
:10118000240801968770B7CFDF91CF911F910F91FF
:10119000FF90EF9008959F92AF92BF92CF92DF920F
:1011A000EF92FF920F931F93CF93DF93CDB7DEB7EC
:1011B00061970FB6F894DEBF0FBECDBF8C0185E0FE
:1011C000F801DE011D9601900D928A95E1F7D80194
:1011D0001296EC9090919B01E0919C0120919E01D0
:1011E00030919F012115310531F0EF3F31F481E05D
:1011F0009F3F19F403C081E001C080E0B82FB170B7
:101200009B2E80FD47C1D8014C9111965C9111979E
:101210001396AD90BC9014978BE9C82E81E0D82E20
:10122000F0909D01B501621B730B2091000130917C
:101230000101FF2009F4D9C08091A0016217730752
:1012400008F095C0282F207F09F052C05E1313C00C
:10125000491311C0FE2CE1100EC08F708061809385
:10126000A0010E944508C6010E94C7058091A00107
:10127000F80185834DC1AB2831F05F3F31F481E047
:101280004F3F19F403C081E001C080E080FD03C03E
:1012900081E08E2502C080E090E0F82FF170FF2EF3
:1012A00080FF1CC08091690120916A0136E082179D
:1012B00009F40BC190E0389FF001399FF00D112423
:1012C000E559FE4F6181561306C06081461303C085
:1012D0006281E61203C001968770E9CFFE2CEE20F2
:1012E00009F416C18091A00181608093A00154C0CF
:1012F0005E1306C0491304C0E11002C0F80199C092
:10130000C8010E942606882361F1EE2051F1209148
:10131000A001822F82958F7090E0029774F08091E7
:101320009B0190919C0198878F831986BB86AA8622
:101330002C87CE0107960E94C70586E0F801ABE92D
:10134000B1E001900D928A95E1F70E9453080E9446
:1013500045080AC05E1711F1C8010E9426068111D6
:101360002CC0C8010E94C705FF24F394D1C0282FC8
:10137000207F81F77A2DB98AA88A6E2D89890E94EB
:101380002E068BE991E00E94C70586E0D6011D92EA
:101390008A95E9F70E944508F12CBAC04913DCCFC1
:1013A000E110DACFF8018583C8010E94C70586E005
:1013B000D6011D928A95E9F7ABC0EE2091F22091FB
:1013C000A001822F82958F7090E002970CF4B5CF28
:1013D00080919B0190919C019A8389831B82BD829D
:1013E000AC822E83CE010196A6CF6217730708F058
:1013F00044C0FE2CEE2009F4B4CF5E1330C0491374
:101400002EC02091A00120FD21C0822F82958F70D7
:10141000482F50E041155105C9F0F80125834F30A0
:10142000510541F08F5F982F9295907F822F8F709A
:10143000892B8583C8010E94C70586E0F801ABE9C6
:10144000B1E001900D928A95E1F73CC086E0F80189
:10145000ABE9B1E001900D928A95E1F759C0C8015E
:101460000E942606811169CF8091A001816080933E
:10147000A001C8010E94C7054BC07A2DB98AA88A6D
:101480006E2D89890E942E0686E0D6011D928A95CE
:10149000E9F718C0EE2009F464CFC8010E942606BF
:1014A000F82E882309F45DCF86E0F801ABE9B1E0BE
:1014B00001900D928A95E1F78BE991E00E940F036C
:1014C0000E9453080E94450823C04D875E878D8582
:1014D0009E850E94F607292F22952F70223028F42E
:1014E0009F7039F0811105C00BC0243028F49F7023
:1014F00049F4805E883020F0C8010E94C7059F2C07
:10150000F92C06C0D80115969C91907F91F7F8CFE1
:101510008F2D61960FB6F894DEBF0FBECDBFDF9161
:10152000CF911F910F91FF90EF90DF90CF90BF90E0
:10153000AF909F9008951F93CF93DF93CDB7DEB701
:101540002C970FB6F894DEBF0FBECDBF4F835887E0
:1015500069877A878B879C87CE0107960E94CB0884
:101560008823D1F09F8188852A853B85232B31F004
:101570008F3F31F481E09F3F19F403C081E001C047
:1015800080E080FD47C04F81588569857A858B85CD
:101590009C850E943D063EC086E0FE013796DE0136
:1015A000119601900D928A95E1F7FF81E8856A8591
:1015B0007B856115710531F0EF3F31F481E0FF3F2C
:1015C00019F403C081E001C080E080FD23C02091B8
:1015D0006A0130E0C901019687709927409169013D
:1015E00050E084179507F1F1F983EA837D836C83DA
:1015F00096E0929FD001939FB00D1124A559BE4F44
:10160000FE01319601900D929A95E1F780936A015F
:101610000E94240816E08091690190916A0189175F
:1016200071F1189FC001112485599E4F0E94CB086B
:10163000882329F1E09169011E9FF0011124E559E9
:10164000FE4F4081518162817381848195810E9426
:101650003D068091690190E00196877099278093FB
:101660006901D9CF0E94070610926A0110926901A0
:10167000EBE9F1E086E0DF011D928A95E9F72C960F
:101680000FB6F894DEBF0FBECDBFDF91CF911F9193
:1016900008958091C10185958595859508958091DE
:1016A000C101877008959091C101977081E009F49C
:1016B00080E008958091E40108959091E401892BE0
:1016C0008093E401089580959091E40189238093AB
:1016D000E40108951092E40108959091E301892BAB
:1016E0008093E301089580959091E301892380938D
:1016F000E30108951092E30108958091C2010895D5
:1017000008950C94800B0C94810B90912D0292FD06
:1017100008C09091C201981721F08093C2010C94E7
:10172000830B08958091C201882329F01092C20191
:1017300080E00C94830B0895CF93DF93E091020136
:10174000F09103018091E4018083E0910201F09126
:10175000030190818091E301892B80838091C201F4
:10176000882381F0E0910201F09103019081892B9F
:10177000808380910201909103010E94BB1481112A
:101780000E94920BC0910201D091030140E250E00F
:1017900061EA71E0CE010E94341D892B69F080E27C
:1017A000FE01A1EAB1E001900D928A95E1F7CE0128
:1017B000DF91CF910C947514DF91CF9108950C9423
:1017C000800B90912D0292FD10C098E0899F9001AE
:1017D0001124262B2093C1010E94BF068091C101D4
:1017E0008595859585950C94DF0B0C94BF0610921A
:1017F000C10180E00C94DF0B2091C1018095822310
:101800008093C101982F977099F430E0482F082EEB
:10181000000C550B2417350759F090912D0292FDBD
:1018200007C08595859585950E94E0060C94F70B79
:10183000089590912D0292FB222720F9281769F034
:1018400080FB92F990932D0280912C0290912D02B1
:101850000E94670C82E00C94FC0B089580912D028D
:1018600082FB882780F991E089270C94190C81E08C
:101870000C94190C80E00C94190C6FEF7FEF80E052
:1018800090E00C946D1D80E090E00E94491D21E0E5
:10189000893E9E4F09F020E0822F089582E090E07B
:1018A0000C94411D83E090E00C94411DCF9384E0A3
:1018B00090E00E94411DC82F82E290E00E94411DED
:1018C0002C2F30E0A901582BCA01CF910895CF9356
:1018D000C92F682F84E090E00E944F1D6C2F82E298
:1018E00090E0CF910C944F1DAB01BC018FE090E0D4
:1018F0000C94611DAB01BC0183E190E00C94611D6F
:1019000060E070E0CB010C947A0C60E070E0CB01F9
:101910000E94740C0C94800C69EE7EEF80E090E0E5
:101920000E946D1D60E082E090E00E944F1D60E02B
:1019300083E090E00E944F1D1092650110926601B5
:10194000109267011092680160E084E090E00E94CC
:101950004F1D60E082E290E00E944F1D60E085E054
:1019600090E00E944F1D60E086E090E00E944F1DD5
:101970006FEF87E090E00E944F1D40E050E0BA0119
:1019800088E090E00E94611D60E08DE090E00E94A0
:101990004F1D40E050E0BA0188E190E00E94611DD7
:1019A00060E087E190E00E944F1D40E050E0BA0106
:1019B0008CE190E00E94611D60E070E080E290E0C8
:1019C0000E946D1D40E050E0BA0188E190E00E9465
:1019D000611D0C94850C0C948C0C682F8EE090E0AB
:1019E0000C944F1D0E9421166093F5017093F6012F
:1019F0008093F7019093F8016093F1017093F201E5
:101A00008093F3019093F401089585B7806885BFB2
:101A100085B7806885BF089581E008950C940C0D0A
:101A200008950C94100D0C94100D0C94130D0C943F
:101A3000100D0C94170D0C94100D0E94050D8DEADD
:101A40009FE00E945F140E941B0D0C94190D0E94D0
:101A5000110D0C94100D0E94C70F0C94A9020E9446
:101A60000C160E94AC100E942B0D0C94150D5F9269
:101A70006F927F928F929F92AF92BF92CF92DF929E
:101A8000EF92FF920F931F93CF93DF93CDB7DEB703
:101A90002A970FB6F894DEBF0FBECDBF0E94C110CB
:101AA000C82E81110E94F20C35EE832E31E0932E68
:101AB00000E010E0502E802F0E94EB0F5C01F4013B
:101AC000619071904F016826792661147104B1F418
:101AD0000F5F1F4F0630110569F78FEF89838A83E7
:101AE0001B820E9415168160782F9D838C8349810B
:101AF0005A816B818D810E94C5023AC08091F901A3
:101B000081FD0E94F40FD12CEE24E394F12CC3014B
:101B10008E219F21892B29F10E940E0D8823A9F087
:101B2000DE825F82AE20BF2081E0AB2809F480E036
:101B300088870E9415168160782F9A8789874E8141
:101B40005F8168858A850E94C502000F111FF80118
:101B5000EB51FE4F80819181E826F926F182E082E7
:101B600007C0D394EE0CFF1CFEE0DF12D0CFB0CF45
:101B700081E0C11001C080E02A960FB6F894DEBF64
:101B80000FBECDBFDF91CF911F910F91FF90EF90CE
:101B9000DF90CF90BF90AF909F908F907F906F908D
:101BA0005F9008950E94370D0C94BA02CF93DF9393
:101BB0000E94D60EEC01811523E59207A0F5811550
:101BC00032E5930708F09EC0811540E29407C0F407
:101BD000811551E0950708F0CDC0853A910550F484
:101BE0008430910508F0C6C0019709F0C0C081E0BB
:101BF00090E0C1C0805E9109089708F4BBC0B7C0EF
:101C0000C11581E5D80708F077C0C11520E5D207D6
:101C100008F051C0C11530E4D30708F4A8C0DF7044
:101C2000CE01906AA8C0811546E5940700F581159C
:101C300055E5950708F081C0C11584E5D80708F07F
:101C400076C0CE018370992721E030E002C0220FD8
:101C5000331F8A95E2F79C2F9695969540E2949FC4
:101C6000E0011124C22BD32BCE019A6884C08115C8
:101C70002AE5920780F4811539E5930708F066C0DC
:101C8000811548E5940708F472C0D82FCC27CE01FF
:101C9000806F906A70C090568115904208F067C0BE
:101CA0008D2F8F710E946A0FDD27D0628F71AE0178
:101CB000582BCA0160C0CE0174E0969587957A953D
:101CC000E1F7282F23703C2F337081E090E002C0B1
:101CD000880F991F3A95E2F79C68AC01522B9A0144
:101CE0009C2F9F709695969550E2959FE001112448
:101CF000C9018C2B9D2B3FC0DC2FCC27CE01816FDF
:101D0000906A39C08370992721E030E002C0220F29
:101D1000331F8A95E2F79C2F9695969580E2989FBF
:101D2000E0011124C22BD32BCE019C6824C0DC2FF0
:101D3000CC27CE01846F906A1EC00E946A0F8F71FB
:101D400090E0D82FCC27CE01906215C08F700E94F2
:101D50006A0F94E0D695C7959A95E1F7CF70D0E0D9
:101D6000DC2FCC27D0699E01282BC90104C080E05C
:101D700090E001C0CE01DF91CF91089524E5829FCC
:101D8000C0011124FC012EE0729FE00DF11D112411
:101D9000E60FF11DEE0FFF1FEE5BFE4F8591949154
:101DA00008950E94BE0E0E94D60D089582389105B6
:101DB00069F1B0F48133910509F46DC048F48932BA
:101DC000910509F463C08A32910509F469C0089548
:101DD0008533910509F455C089339105B9F008950B
:101DE000833E910569F138F4803E9105B1F0823E61
:101DF000910509F10895863E9105A9F1873E910567
:101E0000B9F1843E910509F064C023C020912C02F1
:101E100020FD4FC021FD4DC0089580912C0280FD12
:101E200044C080912D0280FF44C080912C0284FD2B
:101E300042C083EE4DC080912C0282FF38C0F5CFA6
:101E400080912C0282FD33C080912D0280FD31C033
:101E5000ECCF80912D0281FF32C080912C0284FD55
:101E60002AC087EE35C080912C0283FF26C0F5CFB3
:101E700080912C0283FD21C080912D0281FD1FC025
:101E8000ECCF80912C0285FD1CC01DC080912C02DE
:101E900085FD19C016C080912C0286FD16C017C0A2
:101EA00080912C0286FD13C010C089E311C082EE20
:101EB0000FC080EE0DC080E00BC086EE09C084EE3E
:101EC00007C089E205C085E303C08AE201C081E35F
:101ED00090E0089590912C0292FF0DC0282F287158
:101EE000283019F4877F846006C0282F247124309D
:101EF00011F48B7F886093FF0DC0282F2871283143
:101F000019F4877E846106C0282F2471243111F4CE
:101F10008B7E886120912D0220FF0DC0382F3871F3
:101F2000383019F4877F816006C0382F3171313025
:101F300011F48E7F886021FF0DC0282F2871283171
:101F400019F4877E816106C0282F2171213111F497
:101F50008E7E886194FD877E089580E008950C94BC
:101F60003D0C0E94C1108FE39CE90197F1F700C07E
:101F700000000E94C11080E00E94EB0F80FF04C0AF
:101F80000E94AF0F0C94621608950C94B10F0E943A
:101F9000430C811102C00E94EB0C0E944E0C8093F6
:101FA000F9010E94560C90932D0280932C020E94FE
:101FB000C50F0E94520C682F70E080E090E00E94F4
:101FC0005F0660916101709162018091630190915F
:101FD00064010C949706E82FF0E0EE0FFF1FE65C1B
:101FE000FD4F808191810895089580EA8A95F1F7E7
:101FF000089500C008950C94F50F08950C94FD0FFA
:102000000C94FE0F0C94FD0F0C940210F894E82F22
:10201000E295EF70F0E031A1282F2F7081E090E081
:1020200001C0880F2A95EAF7982F9095932391A3E2
:1020300092A1892B82A3789408950F931F93CF9335
:10204000DF93CFE1D1E089918F3F11F00E9406101C
:1020500081E0C532D807B9F7C1E1D1E00FE111E065
:1020600089918F3F11F00E9406100C171D07C1F7D0
:10207000DF91CF911F910F910895BF92CF92DF9280
:10208000EF92FF920F931F93CF93DF938C01C62F94
:10209000D0E0CE01815E9E4F6C01FC0190819F3F9C
:1020A00009F450C0B62EF894E92FE295EF70F0E0F5
:1020B00081A19F7021E030E001C0220F9A95EAF7DC
:1020C000822B81A382A12095282322A378940E94A9
:1020D000F90FE1E1F1E04FE151E021E030E0E12CE6
:1020E000F12C61916F3F89F0A62FA295AF70B0E0FF
:1020F00090968C9190E06F7002C0959587956A9547
:10210000E2F780FD02C0C90102C080E090E0E82A49
:10211000F92A220F331F4E175F0719F7F601808146
:102120008F3F11F00E94061061E0E114F10409F400
:1021300060E08B2D0E94FB0FCC0FDD1FC00FD11F65
:10214000F982E882DF91CF911F910F91FF90EF907C
:10215000DF90CF90BF9008950E941D108CE0EAE3BD
:10216000F2E0DF01982F1D929A95E9F7EEE2F2E096
:10217000DF011D928A95E9F786E00E940C110C940C
:102180003402FF920F931F93CF93DF93CDB7DEB747
:102190002C970FB6F894DEBF0FBECDBF8E010F5F38
:1021A0001F4F8CE0F80111928A95E9F7F12C6F2D01
:1021B000C8010E943D10F394F6E0FF12F8CF4CE006
:1021C00050E0B8018EE292E00E94341DFF24F394A7
:1021D000009709F4F12C892B41F08CE0F801AEE274
:1021E000B2E001900D928A95E1F72F2D46E06AE367
:1021F00072E08EE292E00E940D110E9436028F2D55
:102200002C960FB6F894DEBF0FBECDBFDF91CF91F5
:102210001F910F91FF9008950895FF920F931F93C0
:10222000CF93DF93F82E092F162FD72FC42F2223F9
:1022300049F081E08093FC010E9415169093FB0108
:102240008093FA018091FC018823D9F08091FA01F2
:102250009091FB010E942D16059798F0EF2DF02F1D
:10226000A12FBD2F80E090E04C2F50E08417950700
:1022700034F4219131912D933D930196F7CF109233
:10228000FC01DF91CF911F910F91FF9008950E9463
:10229000EA170E942F0D0C94F6170E94FA170E945D
:1022A000D20D0C9414180E94B3150E94D1170E94ED
:1022B0001D0D0E9447110E944D110E94270DFBCF5A
:1022C000CF93DF93EC01FB018281882309F43CC1A9
:1022D000C430FDE5DF0760F4CB3F9CE5D90788F407
:1022E0009E0122503C452431310508F02EC109C021
:1022F000C236EDE5DE0729F0C63AFDE5DF0709F055
:1023000024C10E94560C90932D0280932C02C1315F
:102310008CE5D80709F4C6C008F042C0C930ECE526
:10232000DE0709F49BC000F5C5308CE5D80709F439
:1023300085C078F4C330ECE5DE0709F478C008F016
:102340007AC0C230DC4509F0F5C080912C02816072
:10235000EFC0C7309CE5D90709F478C008F07AC00F
:1023600080912C028061E4C0CD30FCE5DF0709F4E8
:1023700087C058F4CB309CE5D90709F479C008F040
:102380007BC080912C0288606FC0CF30FCE5DF07F6
:1023900009F480C008F082C080912C02877FC8C0F9
:1023A000CE3F9CE5D90709F471C000F5C531FCE5C5
:1023B000DF0709F485C068F4C3319CE5D90709F447
:1023C00075C008F095C00E94070680912C028F7797
:1023D000AFC0CC3FFCE5DF07A9F108F054C0CB3F0C
:1023E000DC4509F0A7C080912D0240C0C230EDE568
:1023F000DE0709F489C058F4C1158DE5D80709F442
:102400005AC008F069C080912D0282602FC0C23688
:10241000EDE5DE0709F47CC0C63AFDE5DF0709F407
:1024200081C0C330DD4509F085C080E06EC0809179
:102430002C0282607DC080912C0216C080912C02FB
:10244000886076C080912D0282604FC080912C02FE
:1024500080626EC080912C0280646AC00E94070670
:1024600080912C02806864C0846062C081603DC03D
:1024700080912C028E7F5CC080912C028D7F58C091
:1024800080912C0216C080912D0218C080912D02DF
:102490008D7F2BC080912C028F7E4AC080912C02B0
:1024A0008F7D46C080912C028F7B42C080912C0290
:1024B000877F8B7F3DC080912D028D7F8E7F15C0E1
:1024C00080912C0282FB222720F991E0922790FB39
:1024D00082F990FB83F92CC080912D02982F909562
:1024E00091708E7F892B90FB81F980932D0222C001
:1024F0000E94070680912C0287FB222720F991E099
:10250000922790FB87F914C081E00E94ED0C12C065
:1025100080912C0284FB222720F991E0922790FBE6
:1025200084F906C080912C02982F909590FB80F939
:1025300080932C0280912C0290912D020E94670CB6
:102540000E94070680E001C081E0DF91CF910895ED
:102550000F931F9341E050E060E070E08A019B011F
:1025600004C0000F111F221F331F8A95D2F7C90123
:10257000B8010E945F061F910F910C940706482F27
:1025800050E0FA013597EF33F10508F060C0E85AE2
:10259000FF4F0C942B1D0E94EB0C55C08091F9014C
:1025A000817F8E7F8093F90181E08093FD01089502
:1025B0000E94390248C08091F901982F909591703E
:1025C00090FB80F98093F90191113DC0897F877F4D
:1025D00010C08091F90181FB222720F991E0922718
:1025E00090FB81F98093F901992369F18091F901B8
:1025F00081608093F90127C08091F90182FB222735
:1026000020F991E0922790FB82F9ECCF8091F901BB
:1026100083FB222720F991E0922790FB83F9E2CFF8
:102620000E94070680912C0287FB222720F991E067
:10263000922790FB87F980932C0205C0895301C033
:102640008D510E94A81281E0089580E0FACF80E0C9
:10265000089580E008950C942913CF93C82F80919A
:10266000FD01882319F0813031F02BC00E945A0BF4
:10267000823249F504C00E945A0B823261F48C2FD9
:102680000E942B13811104C08C2F0E94BF1217C00F
:1026900081E090E014C08C2F0E94291381110EC09C
:1026A000C43149F018F4CB3049F00FC0C93219F0E9
:1026B000C83321F00AC01092FD0107C081E081708B
:1026C00006C01092FD0180E002C080E0F8CFCF91FB
:1026D0000895CF93DF9386319C4541F5EB010E942D
:1026E0005A0B982F8A81209102013091030188238F
:1026F00079F09A7A81E009F480E08093FE019111EB
:1027000002C069E201C065E3C9010E9451150AC017
:102710008091FE01811102C069E201C065E3C90137
:102720000E945C150E949C0B80E001C081E0DF915B
:10273000CF9108950F931F93CF93DF93C42FD22F80
:10274000FC0182818823C9F0409301020E94151682
:10275000909300028093FF0180E28C0F883008F094
:1027600057C0C77081E001C0880FCA95EAF7DF91B2
:10277000CF911F910F910C949903809101024813FE
:1027800030C08091FF01909100020E942D16883C7C
:10279000910538F510E21D0FCD17B9F080E28C0FCE
:1027A000883040F4C77081E001C0880FCA95EAF70D
:1027B0000E94A003183028F581E09D2F977001C07A
:1027C000880F9A95EAF70E949903802F0E94900340
:1027D0001830F0F4D77081E001C0880FDA95EAF77D
:1027E0000AC080E28C0F883098F4C77081E001C085
:1027F000880FCA95EAF7DF91CF911F910F910C9442
:10280000A003802FDF91CF911F910F910C94900323
:10281000DF91CF911F910F9108950F939C01CB01F0
:10282000243F4CE5340731F188F4293DFCE53F07AE
:10283000D9F02A3D4CE5340779F1283D3C45A9F50E
:1028400006E221EE41EE68ED7CE52BC0263FFCE57B
:102850003F07E1F0A8F0273F3C4539F507E225EEB8
:1028600046EE67EF7CE51DC007E225EE45EE69ED1B
:102870007CE517C006E221EE40EE64EF7CE511C076
:1028800007E225EE44EE65EF7CE50BC006E221EEA3
:1028900042EE66EF7CE505C008E221E045EE6AED18
:1028A0007CE50E949A1380E008C0FC0182818823A5
:1028B00019F01092010201C081E00F9108959093E8
:1028C00027018093260108959093070280930602C2
:1028D0000895E0910602F0910702309721F00190EF
:1028E000F081E02D099480E00895E0910602F091D6
:1028F0000702309799F020911001222359F020917E
:102900002C0227FF07C0DC012C9111962C93119704
:1029100026E02C930280F381E02D09940895209104
:102920000402309105022817390771F090930502CF
:1029300080930402E0910602F0910702309721F0A3
:102940000680F781E02D09940895209102023091CC
:1029500003022817390771F0909303028093020253
:10296000E0910602F0910702309721F00084F18592
:10297000E02D09940895FC0132968091100188237E
:1029800031F080912C0287FF02C09EE101C096E0E9
:1029900080E0915028F021912223D9F38F5FF9CF65
:1029A0000895662351F1209110012223E9F020912E
:1029B0002C0227FF19C0462F4695469546954E3165
:1029C000E0F4677021E030E002C0220F331F6A9507
:1029D000E2F7FC01E40FF11D828190E02823392306
:1029E00081E0232B69F409C0FC01329608962191FD
:1029F000621729F0E817F907D1F780E0089581E020
:102A000008959C01FC0132969FEF80E041914617AA
:102A100089F09F3F19F4411101C0982F8F5F8630D4
:102A2000A9F79F3F39F0F901E90FF11D97FDFA95DC
:102A30006283089508959C012A5F3F4FFC01428103
:102A4000461301C01282019682179307B9F70895C1
:102A5000262F2695269526952E3168F4FC01E20F47
:102A6000F11D677021E030E001C0220F6A95EAF79E
:102A70008281282B22830895262F26952695269538
:102A80002E3170F4FC01E20FF11D677021E030E09F
:102A900001C0220F6A95EAF72095828128232283BC
:102AA000089520911001222329F020912C0227FD66
:102AB0000C9428150C94011520911001222329F063
:102AC00020912C0227FD0C943C150C941B15209191
:102AD0001001FC013296222331F080912C0287FFF5
:102AE00002C08EE101C086E0DF011D928A95E9F700
:102AF000089508950C94791583E0809308020C944E
:102B00007A15811102C081E001C082E08093080241
:102B10000C947A150C94811581E0809308020C9432
:102B20007A150C948C1508950C9493150C949415A7
:102B30000C9493150C9493150C949315CF930E94B9
:102B40009A150E94C1100E949815C0E08C2F0E9417
:102B5000EB0F892B29F4CF5FC630C1F780E001C0AD
:102B600081E0CF91089508951F920F920FB60F92B2
:102B700011248F939F93AF93BF938091090281118A
:102B800013C08091460290914702A0914802B091F3
:102B900049024196A11DB11D8093460290934702C0
:102BA000A0934802B0934902BF91AF919F918F913A
:102BB0000F900FBE0F901F90189580914E02843099
:102BC00031F10E949A021092090220E488E190E01B
:102BD0000FB6F894A895809360000FBE2093600014
:102BE00083B7817F846083BF83B7816083BF78941C
:102BF000889583B78E7F83BF0FB6F894A895809190
:102C00006000886180936000109260000FBE08959C
:102C10000E9407060C949E0282E084BD93E095BD5D
:102C20009AEF97BD80936E0008952FB7F894809126
:102C3000460290914702A0914802B09149022FBFED
:102C400008952FB7F89460914602709147028091E1
:102C50004802909149022FBF08959C014FB7F89404
:102C60008091460290914702A0914802B09149029A
:102C70004FBF821B930B089578941F920F920FB64B
:102C80000F9211248F939F93AF93BF93809146022D
:102C900090914702A0914802B09149020196A11D6E
:102CA000B11D8093460290934702A0934802B093CF
:102CB0004902BF91AF919F918F910F900FBE0F90DE
:102CC0001F901895F89481E08093E00080E2809353
:102CD000D800E9ECF0E010828FE19EE40197F1F773
:102CE00000C000001DBA109268001CBC10BE1FBAC4
:102CF00010927A0010926E0010926F001092700085
:102D00001092710010821092BC0011B814B817B85C
:102D10001AB81DB810BA12B815B818B81BB81EB832
:102D200011BA0C9400FE089580912A020895089526
:102D30000895CF93DF9320911001222339F0209141
:102D40002C0227FF03C060E222E002C068E021E01D
:102D50002093E9002FEF3091E800215035FD06C0A7
:102D600035ED3A95F1F700002111F5CF2091E800FB
:102D700025FF1DC0EC0180911001811105C040E0CC
:102D800050E068E070E003C070E040E050E0CE0149
:102D90000E9486188091E8008E778093E80080E298
:102DA000FE01AAE0B2E001900D928A95E1F7DF9171
:102DB000CF9108950895089580914D02811109C021
:102DC0000E94131A0E94751A8091E2008460809319
:102DD000E200089510924D0208950C9491156091AF
:102DE0004A0281E0611101C080E00C947C15909151
:102DF0004E0281E0943009F080E060914A020C9428
:102E0000811542E061EC81E00E948C1942E261ECA4
:102E100082E00E948C1990914E0281E0943009F07A
:102E200080E060914A020C948A15809150028330B0
:102E300009F45FC030F4813071F0823009F498C039
:102E400008958A3009F484C08B3009F46AC089304F
:102E500009F0A6C020C080914F02813A09F0A0C0BD
:102E60008091E800877F8093E800809153029091E1
:102E70005402892B21F460E28AE092E003C060E012
:102E800080E090E070E00E94D1188091E8008B779C
:102E90008093E800089580914F02813209F080C04C
:102EA0008091530290915402029708F079C080916A
:102EB000E800877F8093E8008091E80082FD05C0EC
:102EC00080914E028111F8CF6BC08091F2009091F9
:102ED000F300029731F48091F100813011F08630D7
:102EE00021F48091F10080932A028091E8008B7791
:102EF00053C080914F02813A09F052C08091530231
:102F000090915402892B09F04BC08091E800877F93
:102F10008093E8008091E80080FFFCCF8091100151
:102F200036C080914F028132D9F580915302909141
:102F30005402892BA9F58091E800877F8093E800EF
:102F40000E94C11980915102809310010C940706D0
:102F500080914F02813221F58091E800877F809334
:102F6000E8000E94C1198091520280932B020895BB
:102F700080914F02813AA1F48091E800877F80938D
:102F8000E8008091E80080FFFCCF80912B028093C5
:102F9000F1008091E8008E778093E8000C94C119CD
:102FA000089584B7877F84BF0FB6F894A895809161
:102FB0006000886180936000109260000FBE90E016
:102FC00080E80FB6F89480936100909361000FBE83
:102FD0000C948C150E94131A0E94751AE2EEF0E010
:102FE00080818460808378940C94101D84E091E04B
:102FF0000C94641480914E028530A9F480914E02A5
:10300000853079F40E94DD1580914C028823B1F35C
:103010000E949E15882391F30E9470180E94070653
:10302000EDCF0C940816089508950C941718292FC5
:10303000332723303105C9F060F42130310581F0A8
:103040002230310509F044C08BE390E02AEB32E0F6
:1030500043C021323105E1F02232310549F138C057
:1030600082E190E025EF32E037C099278130910569
:1030700049F028F0029761F5E2E9F2E005C0E6EBDD
:10308000F2E002C0E0EAF2E0849190E09F0124C007
:103090006115710541F061307105D1F489E090E06E
:1030A00025EE32E019C089E090E02CEC32E014C04B
:1030B0006115710541F06130710551F48BE390E0C9
:1030C00027E033E009C080E490E022E433E004C06C
:1030D00080E090E020E030E0FA0131832083089521
:1030E00084E189BD86E189BD09B400FEFDCF8091F0
:1030F000D8008F7D8093D8008091E000826080931B
:10310000E0008091E00081FDFCCF0895CF92DF9236
:10311000EF92FF920F931F93CF93DF93EC018B01FC
:103120007A010E94E019811133C0E114F10439F0F1
:10313000F70180819181081B190BC80FD91FC12C81
:10314000D12C0115110519F18091E80085FD16C0FB
:103150008091E8008E778093E800E114F10449F053
:10316000F70180819181C80ED91ED182C08285E08D
:103170000FC00E94E019882321F30AC0899180932F
:10318000F10001501109FFEFCF1ADF0ADACF80E01A
:10319000DF91CF911F910F91FF90EF90DF90CF9033
:1031A000089520915502309156022617370748F0AE
:1031B0006115710539F42091E8002E772093E8001D
:1031C00001C0B901FC0120E06115710569F1809130
:1031D0004E028823E1F18530E1F18091E80083FD22
:1031E0003AC08091E80082FD2CC08091E80080FF09
:1031F000EBCF8091F2009091F3006115710551F0D1
:103200008830910538F421912093F10061507109C3
:103210000196F3CF21E0089709F020E08091E800C3
:103220008E778093E800D0CF2111D1CF0AC0809152
:103230004E02882361F0853061F08091E80083FDC3
:103240000AC08091E80082FFF2CF80E0089582E01A
:10325000089583E0089581E008952091550230910A
:1032600056022617370748F06115710539F4209189
:10327000E8002E772093E80001C0B901FC0120E0AE
:103280006115710581F180914E02882309F43EC0D9
:10329000853009F43DC08091E80083FD3BC08091FA
:1032A000E80082FD2DC08091E80080FFE9CF809189
:1032B000F2009091F3006115710559F08830910585
:1032C00040F424912093F1003196615071090196E8
:1032D000F2CF21E0089709F020E08091E8008E7796
:1032E0008093E800CDCF2111CECF0AC080914E024D
:1032F000882361F0853061F08091E80083FD0AC089
:103300008091E80082FFF2CF80E0089582E0089586
:1033100083E0089581E00895982F973068F59093A1
:10332000E900981739F07091EC002091ED00509170
:10333000F00003C0242F762F50E021FD02C09F5FD4
:10334000ECCF3091EB003E7F3093EB003091ED00FD
:103350003D7F3093ED003091EB0031603093EB0016
:103360007093EC002093ED005093F0002091EE005C
:1033700027FDE5CF80E008958F708093E90081E01C
:10338000089580914F0287FF11C08091E80082FD6F
:1033900005C080914E028111F8CF11C08091E800E4
:1033A0008B770BC080914E02882349F08091E80012
:1033B00080FFF8CF8091E8008E778093E800089531
:1033C0002091E4003091E50095E64091EC00842FD7
:1033D000817040FF23C08091E80080FD1DC0809176
:1033E0004E02882399F0853099F08091EB0085FD9D
:1033F00011C04091E4005091E5002417350729F3EE
:10340000915011F09A01E1CF84E0089582E008958F
:1034100083E0089581E0089580E008954091E800F8
:1034200042FFDDCF08950E94841A0E948C1AE0EEBC
:10343000F0E0808181608083E8EDF0E080818F772B
:10344000808319BCA7EDB0E08C918E7F8C93808136
:103450008F7E808310924D0208950F931F93CF9318
:10346000DF930E94841A0E948C1AC8EDD0E08881F4
:103470008F77888388818068888388818F7D88831F
:10348000E7EDF0E080818068808319BC10924E02E5
:1034900010924A0210924C0210924B0200EE10E081
:1034A000F80180818B7F808388818160888342E0FE
:1034B00060E080E00E948C19E1EEF0E080818E7F78
:1034C0008083E2EEF0E0808181608083808188608B
:1034D0008083F80180818E7F8083888180618883EA
:1034E000DF91CF911F910F910895E8EDF0E0808179
:1034F0008F7E8083E7EDF0E080818160808381E0D2
:1035000080934D020C942D1AE8EDF0E080818C7FC1
:1035100080831092E20008951092DA001092E10088
:1035200008951F920F920FB60F9211240BB60F92AF
:103530002F933F934F935F936F937F938F939F93BB
:10354000AF93BF93EF93FF938091E10082FF0BC095
:103550008091E20082FF07C08091E1008B7F809321
:10356000E1000E940F1D8091DA0080FF1FC0809152
:10357000D80080FF1BC08091DA008E7F8093DA0034
:103580008091D90080FF0DC084E189BD86E189BDAD
:1035900009B400FEFDCF81E080934E020E94DC164C
:1035A00005C019BC10924E020E94EA168091E100FB
:1035B00080FF19C08091E20080FF15C08091E20079
:1035C0008E7F8093E2008091E20080618093E20030
:1035D0008091D80080628093D80019BC85E08093E8
:1035E0004E020E94EF168091E10084FF30C080916E
:1035F000E20084FF2CC084E189BD86E189BD09B465
:1036000000FEFDCF8091D8008F7D8093D8008091FF
:10361000E1008F7E8093E1008091E2008F7E8093B5
:10362000E2008091E20081608093E20080914A0292
:10363000882311F084E007C08091E30087FD02C079
:1036400081E001C083E080934E020E94F7168091D2
:10365000E10083FF29C08091E20083FF25C08091B3
:10366000E100877F8093E10082E080934E02109218
:103670004A028091E1008E7F8093E1008091E20018
:103680008E7F8093E2008091E20080618093E2006F
:1036900042E060E080E00E948C198091F000886038
:1036A0008093F0000E94ED16FF91EF91BF91AF91D2
:1036B0009F918F917F916F915F914F913F912F914A
:1036C0000F900BBE0F900FBE0F901F9018951F927A
:1036D0000F920FB60F9211240BB60F922F933F93B8
:1036E0004F935F936F937F938F939F93AF93BF930A
:1036F000CF93DF93EF93FF93C091E900CF70809158
:10370000EC00D82FD17080FDD0E81092E9008091B4
:10371000F000877F8093F00078940E94AF1B109296
:10372000E9008091F00088608093F000CD2BCF708D
:10373000C093E900FF91EF91DF91CF91BF91AF91DD
:103740009F918F917F916F915F914F913F912F91B9
:103750000F900BBE0F900FBE0F901F9018951F93E8
:10376000CF93DF93CDB7DEB7AA970FB6F894DEBF3D
:103770000FBECDBFEFE4F2E08091F100819322E033
:10378000E735F207C9F70E9415178091E80083FF1B
:103790002EC180914F0290915002492F50E04A3043
:1037A000510508F024C1FA01E956FF4F0C942B1D76
:1037B000803821F0823809F01AC108C080914B028C
:1037C00090914C02992389F082600FC0809153023E
:1037D0008F70873008F00BC18093E9008091EB0077
:1037E00085FB882780F91092E9009091E800977F87
:1037F0009093E8008093F1001092F100D1C0282F3F
:103800002D7F09F0F4C0882319F0823061F0EFC0F9
:1038100080915102813009F0EAC0933009F080E0D4
:1038200080934C022EC08091510281112AC0809158
:1038300053028F702FEF280F263008F0D8C08093E6
:10384000E9002091EB0020FF1CC0933021F480910F
:10385000EB00806214C09091EB0090619093EB00BC
:1038600021E030E0A90102C0440F551F8A95E2F71C
:103870004093EA001092EA008091EB008860809308
:10388000EB001092E9008091E800877F8093E800C8
:103890000E94C119ACC08111AAC0109151021F77BA
:1038A0008091E3008078812B8093E3008091E80091
:1038B000877F8093E8000E94C1198091E80080FF13
:1038C000FCCF8091E30080688093E300111102C077
:1038D00082E001C083E080934E0289C0805882302C
:1038E00008F085C080915102909152028C3D53E0C6
:1038F000950779F583E08A838AE289834FB7F89444
:10390000DE01139620E03EE051E2E32FF0E0509319
:103910005700E49120FF03C0E295EF703F5FEF7026
:103920008E2F90E0EA3010F0C79601C0C0968D93BC
:103930009D932F5F243149F74FBF8091E800877F27
:103940008093E8006AE270E0CE0101960E94D118EF
:1039500016C06091530270915402AE014F5F5F4FE9
:103960000E941518BC01892B09F441C09091E80010
:10397000977F9093E80089819A810E942D19809108
:10398000E8008B778093E80032C0803881F5809121
:10399000E800877F8093E80080914A028093F100DD
:1039A0008091E8008E7772CF811121C08091510201
:1039B0009091520299270297D4F48091E800877F72
:1039C0008093E8008091510280934A020E94C119BD
:1039D00080914A02811106C08091E30087FD02C0F8
:1039E00081E001C084E080934E020E940117809123
:1039F000E80083FF0AC08091E800877F8093E80099
:103A00008091EB0080628093EB00AA960FB6F89449
:103A1000DEBF0FBECDBFDF91CF911F9108950895F6
:103A2000CF9380914E028823A1F0C091E900CF701E
:103A30009091EC00892F817090FD80E8C82B109246
:103A4000E9008091E80083FD0E94AF1BCF70C09316
:103A5000E900CF910895EE0FFF1F0024001C0BBE5C
:103A60000790F691E02D0994FB01DC0104C08D91D3
:103A70000190801921F441505040C8F7881B990BE0
:103A80000895F999FECF92BD81BDF89A992780B526
:103A90000895A8E1B0E042E050E00C94751D262F97
:103AA000F999FECF92BD81BDF89A019700B4021634
:103AB00039F01FBA20BD0FB6F894FA9AF99A0FBEE2
:103AC00008950396272F0E94501D0E944F1D252FF9
:103AD0000E94501D242F0C94501D0196272F0E94E8
:103AE000501D0C944F1DDC01CB01FC01F999FECF58
:103AF00006C0F2BDE1BDF89A319600B40D92415076
:0A3B00005040B8F70895F894FFCF85
:103B0A00C800C30194169916DA16DB16971698168A
:103B1A0001676665646261379392363534333231B0
:063B2A00976396959400DC
:00000001FF
